:1000000000308A0081290000FF00030E8301A10057
:100010000A08A0008A010408A2007708A300780853
:10002000A4007908A5007A08A6007B08A70083131E
:1000300083128C308400801E1F288C1A32282208DC
:1000400084002308F7002408F8002508F900260892
:10005000FA002708FB0020088A00210E8300FF0E0B
:100060007F0E09008A110A12ED280A108A100A115F
:1000700082075B345E345F345F345D3460345E34F9
:100080005F345F34613400340A108A100A11820729
:100090000134F634F634F6340134003476347634F0
:1000A0007634893481347E347E347E34BD340034F9
:1000B0007E347E347E3481340034763476347E343B
:1000C0007E340034F634F634FE34FE3481347E342B
:1000D0007634763485340034F734F734F73400342A
:1000E0007E347E3400347E347E34BE347E347E34BE
:1000F0007E3480340034F734F734EB341C3400346D
:100100007F347F347F347F340034FE34F034FE3467
:1001100000340034EF34DF34BF34003481347E34B3
:100120007E347E3481340034F634F634F634F934D7
:1001300081347E347E347E3401340034F634F63437
:10014000F6340934B9347634763476348D34FE346A
:10015000FE340034FE34FE3480347F347F347F3408
:100160008034C034BF347F34BF34C03480347F34F3
:1001700080347F3480341C34EB34F734EB341C345B
:10018000F834F7340734F734F8341E346E347634E8
:100190007A347C34FF34FF34FF34FF34FF341734B7
:1001A00033345534E634F734F034F734F73401346B
:1001B000F7343D345E346E347634793400347E3432
:1001C0007E347E340034F734F734F734F734F734C0
:1001D0008934763476347634893483168601553002
:1001E00083128600BE013E08093C031C002928300A
:1001F0003E0784008C1EFA281A088000BE0AF328E5
:100200008C128A110A121F28393084000008031941
:100210001A290130F800BF30F7006400F70B0D29F0
:10022000F80B0B294A30F700F70B14290000640083
:10023000800B09298A110A124E29F701F8013C089E
:1002400003103D18F707F70CF80CBD18F707F70C6B
:10025000F80C3D19F707F70CF80CBD19F707F70C68
:10026000F80C3D1AF707F70CF80CBD1AF707F70C56
:10027000F80C3D1BF707F70CF80CBD1BF707F70C44
:10028000F80C8A110A1262291F151F1945291E0828
:10029000083C031844290A30B9000429B60136087D
:1002A000093C031C7E29B7013708043C031C722952
:1002B00028303607840041300002BB00BC00053006
:1002C000BD001D29370878074420B9008316860130
:1002D0008312390886006400A630F700F70B6E29F8
:1002E000B70A542983168601FF3083128600640002
:1002F000A630F700F70B7A29B60A4F298A110A129D
:10030000FC2984011F308305673083169900223051
:10031000980090308312980083161F149F141F15A5
:100320009F1107309C00FF308312B40083161F100A
:100330009F141F159F151F1383121F179F178316D6
:100340009F1383121F148316091283129412B4127E
:100350003408831687008312341634088316870006
:100360008312B4113408831687000130831294007D
:100370000030831694000108C739083881000F3017
:10038000F700073083128101813084000008F039C2
:100390000738800064000008F739F719F03977044E
:1003A000800090010030F800920000308316920027
:1003B00007309C00050864000230F700F70BDE29C7
:1003C000000000001C0883120D1383169D018C167B
:1003D000C03083128B040030F8001F08C73978043E
:1003E0009F0083168601FF3083128600B301A801A7
:1003F000A8080319FD2944290C2AB501B6012830A3
:100400008400350884073608352080000038031939
:0C0410000C2AB60AB50AFF29F82963007F
:02400E003D3F34
:00000001FF
